:100000000C9438000C9453000C9453000C9453003F
:100010000C94FE020C940A020C94D1020C94770208
:100020000C94A4020C94DD010C944A020C948A01F5
:100030000C9453000C9453000C9453000C945300F4
:100040000C9453000C9453000C9453000C945300E4
:100050000C9453000000010008004000000100045F
:1000600000000100080020004000800000010004A2
:1000700011241FBECFE5D8E0DEBFCDBF10E0A0E663
:10008000B0E0E4E5FCE002C005900D92A83BB107AA
:10009000D9F710E0A8EBB0E001C01D92A93FB1076D
:1000A000E1F70C9444050C940000089593B7987FF1
:1000B000982B93BF08959EB5987F982B9EBD089569
:1000C00095B5987F982B95BD0895E3B7FF27E77006
:1000D000F070EE0FFF1FEC5AFF4F85919491089539
:1000E000EEB5FF27E770F070EE0FFF1FEC5AFF4FE1
:1000F000859194910895E5B5FF27E770F070EE0FB4
:10010000FF1FE05AFF4F859194910895883040F485
:10011000E82FFF27EE0FFF1FE854FF4F7183608326
:100120000895883040F4E82FFF27EE0FFF1FE854B2
:10013000FF4F118210820895DF92EF92FF920F938A
:100140001F937C01D2B61092CC001092CD00109279
:10015000CE001092CF000E9465009C0144275527D5
:1001600060E074E284EF90E00E940F06293B8DE886
:10017000380786E0480780E0580798F481E1E816E0
:1001800087E2F80670F4B701882799270E94BA051C
:1001900028EE33E040E050E00E94ED0579018A014D
:1001A00023C000271127CA01B90128EE33E040E03F
:1001B00050E00E94ED05C801B7010E94BA057B011D
:1001C0008C0112C08091CC009091CD00A091CE0006
:1001D000B091CF0085B78F7885BF85B7806885BF20
:1001E000889585B78F7785BF8091CC009091CD00A1
:1001F000A091CE00B091CF0022B7BA2FA92F982F8F
:100200008827332744275527822B932BA42BB52BE4
:10021000A80197012D0D311D411D511D8217930716
:10022000A407B50778F21F910F91FF90EF90DF9030
:1002300008951092C8001092C9001092CA0010923E
:10024000CB0008956091C8007091C9008091CA00E8
:100250009091CB0008951092D0001092D10010928E
:10026000D2001092D30008956091D0007091D10017
:100270008091D2009091D3000895893031F48FB5E8
:1002800082608FBD8FB58E7F0AC08A3019F48FB51A
:10029000826002C08FB58D7F8FBD8FB581608FBDAD
:1002A0001BBC1ABC19BC18BC08952FB52E7F2FBDDE
:1002B0002FB522602FBD2EB528602EBD2EB5206132
:1002C0002EBD97BD86BD1BBC1ABC19BC18BC0895B9
:1002D0008FB580688FBD8FB58F7B8FBD08958FB52B
:1002E00080628FBD8FB58F7E8FBD08958FB58F775C
:1002F0008FBD8FB58F7B8FBD08958FB58F7D8FBDDF
:100300008FB58F7E8FBD08959BBD8ABD089599BD21
:1003100088BD08951F920F920FB60F9211242F934C
:100320003F934F935F936F937F938F939F93AF937D
:10033000BF93EF93FF938091C8009091C900A09163
:10034000CA00B091CB000196A11DB11D8093C800D9
:100350009093C900A093CA00B093CB008091CC00C9
:100360009091CD00A091CE00B091CF000196A11D3B
:10037000B11D8093CC009093CD00A093CE00B0939C
:10038000CF008091B8009091B900892B29F0E091BD
:10039000B800F091B9000995FF91EF91BF91AF912D
:1003A0009F918F917F916F915F914F913F912F918D
:1003B0000F900FBE0F901F9018951F920F920FB6BF
:1003C0000F9211242F933F934F935F936F937F93DB
:1003D0008F939F93AF93BF93EF93FF938091BA0056
:1003E0009091BB00892B29F0E091BA00F091BB00FD
:1003F0000995FF91EF91BF91AF919F918F917F915F
:100400006F915F914F913F912F910F900FBE0F9081
:100410001F9018951F920F920FB60F9211242F93D1
:100420003F934F935F936F937F938F939F93AF937C
:10043000BF93EF93FF938091D0009091D100A09152
:10044000D200B091D3000196A11DB11D8093D000C0
:100450009093D100A093D200B093D3008091C200BA
:100460009091C300892B29F0E091C200F091C30064
:100470000995FF91EF91BF91AF919F918F917F91DE
:100480006F915F914F913F912F910F900FBE0F9001
:100490001F9018951F920F920FB60F9211242F9351
:1004A0003F934F935F936F937F938F939F93AF93FC
:1004B000BF93EF93FF938091C6009091C700892B63
:1004C00029F0E091C600F091C7000995FF91EF91E6
:1004D000BF91AF919F918F917F916F915F914F915C
:1004E0003F912F910F900FBE0F901F9018951F9264
:1004F0000F920FB60F9211242F933F934F935F9358
:100500006F937F938F939F93AF93BF93EF93FF93DB
:100510008091BC009091BD00892B29F0E091BC0036
:10052000F091BD000995FF91EF91BF91AF919F911F
:100530008F917F916F915F914F913F912F910F908C
:100540000FBE0F901F9018951F920F920FB60F922B
:1005500011242F933F934F935F936F937F938F93C8
:100560009F93AF93BF93EF93FF938091BE009091C1
:10057000BF00892B29F0E091BE00F091BF000995E2
:10058000FF91EF91BF91AF919F918F917F916F916B
:100590005F914F913F912F910F900FBE0F901F9041
:1005A00018951F920F920FB60F9211242F933F931D
:1005B0004F935F936F937F938F939F93AF93BF936B
:1005C000EF93FF938091C0009091C100892B29F097
:1005D000E091C000F091C1000995FF91EF91BF91AA
:1005E000AF919F918F917F916F915F914F913F91CB
:1005F0002F910F900FBE0F901F9018951F920F9282
:100600000FB60F9211242F933F934F935F936F93E5
:100610007F938F939F93AF93BF93EF93FF938091BB
:10062000C4009091C500892B29F0E091C400F0919D
:10063000C5000995FF91EF91BF91AF919F918F9167
:100640007F916F915F914F913F912F910F900FBECE
:100650000F901F90189583B7887F826083BF12BE6A
:1006600089B7816089BF1092C8001092C9001092AA
:10067000CA001092CB0008958EB5887F83608EBD2E
:100680001DBC1CBC89B7846089BF089585B5887F6F
:10069000846085BD14BC89B7806489BF1092D00086
:1006A0001092D1001092D2001092D3000895E8EB7E
:1006B000F0E011821082329680E0E83CF807C9F73A
:1006C0000E942B030E943C030E94460378940895E5
:1006D0008FB58D7F8FBD8FB58E7F8FBD8FB58F7797
:1006E0008FBD8FB58F7B8FBD8FB58F7D8FBD8FB544
:1006F0008F7E8FBD0895E82FFF27EE0FFF1FEE0FAF
:10070000FF1FEB52FF4F6083477081E090E002C013
:10071000880F991F4A95E2F7818308956A3271051F
:1007200010F46AE270E0E82FFF27EE0FFF1FEE0FD4
:10073000FF1FEB52FF4F6A36710510F069E670E05B
:10074000738362830895E82FFF27EE0FFF1FEE0FDC
:10075000FF1FEB52FF4F828193810895CF93DF9368
:10076000E091D400E43078F4FF27EE0FFF1FEE0F86
:10077000FF1FEB52FF4FA081BB27ED0198A18181A4
:100780008095982398A38091D4008F5F8093D400A4
:10079000843001F1853010F01092D400E091D40043
:1007A000FF27EE0FFF1FEE0FFF1FEB52FF4FA08141
:1007B000BB27ED0188A19181892B88A3E091D4000A
:1007C000FF27EE0FFF1FEE0FFF1FEB52FF4F42817F
:1007D00053810AC04091E7005091E8008091E50004
:1007E0009091E600481B590B2AB58BB59927982F95
:1007F0008827820F911D840F951F292F33272BBD2A
:100800008ABD8091E5009091E600840F951F90933A
:10081000E6008093E5002091E7003091E800821720
:10082000930720F01092E6001092E500DF91CF913F
:10083000089589B78F7E89BF82E00E949100089554
:1008400089B78F7E89BF84E00E945B006EEA73E007
:1008500082E00E948600E5EDF0E020E030E06AE210
:1008600070E0A8E141E050E073836283A083CA0195
:10087000022E02C0880F991F0A94E2F781832F5F2E
:100880003F4F34962430310579F71092E6001092EC
:10089000E50081EB93E09093E8008093E7002AB5B0
:1008A00033278BB52F543C4F9927982F8827820FD9
:1008B000931F292F33272BBD8ABD89B7806189BF3C
:1008C0000895E82FFF27EE0FFF1FEE0FFF1FEB52DB
:1008D000FF4F228133818FEF90E0AC01249FC00154
:1008E000259F900D349F900D1124865D99426FE3F2
:1008F00070E00E94D905CB0199270895282F8FE336
:10090000689FC00111246FEF70E00E94D905665DF9
:100910007F4F6A32710510F46AE270E0E22FFF2720
:10092000EE0FFF1FEE0FFF1FEB52FF4F6A367105F0
:1009300010F069E670E07383628308950F931F934C
:100940000E94200446E06BE181E00E947B0347E0C7
:100950006BE182E00E947B0341E06BE183E00E9457
:100960007B0382EC8ABB83EF8BBB88B38F6088BB31
:1009700082B3806F82BB00E810E01093EB0000931D
:10098000EA0069E181E00E947E041093F000009388
:10099000EF0060E082E00E947E041093F500009377
:1009A000F40067E383E00E947E041F910F91089595
:1009B0008091F1009091F2006091EF007091F00051
:1009C00086179707A9F01092F300681779071CF4AF
:1009D00081E090E002C08FEF9FEF680F791F709366
:1009E000F0006093EF00605882E00E947E0403C034
:1009F00081E08093F3002091EC003091ED00809134
:100A0000EA009091EB0028173907B1F01092EE0040
:100A1000821793071CF421E030E002C02FEF3FEF74
:100A2000820F931F9093EB008093EA0069E9681BA3
:100A300081E00E947E0403C081E08093EE0020915B
:100A4000F6003091F7008091F4009091F50028179E
:100A50003907B1F01092F800821793071CF421E0D7
:100A600030E002C02FEF3FEF820F931F9093F5000D
:100A70008093F40067EB681B83E00E947E04089576
:100A800081E08093F8000895C9E5D8E0DEBFCDBFCE
:100A90000E94570378940E949E04DE011196E1EBB8
:100AA000F0E086E001900D928150E1F78091E9003D
:100AB0008D5F8093E9002CEF3FEF40E050E0EE24A3
:100AC000FF2487018091E9008F5F8093E900215026
:100AD000310941095109B0F78091F3009091EE007E
:100AE00089239091F8008923F1F1A701440F551F44
:100AF0004E0D5F1DFA01EE59FF4FA081EA2FE695DA
:100B0000E695E370FF27EE0FFF1F9E012F5F3F4F1B
:100B1000E20FF31F808191819093F2008093F100A6
:100B2000EA2FE370FF27EE0FFF1FE20FF31F808114
:100B300091819093ED008093EC00A295AF70A3702B
:100B4000BB27AA0FBB1FA20FB31F8D919C9190933F
:100B5000F7008093F600405A5F4FFA01808191813F
:100B60007C01002711270E94D80420E030E440E0F7
:100B700050E0A8CF629FD001739FF001829FE00DEB
:100B8000F11D649FE00DF11D929FF00D839FF00D0C
:100B9000749FF00D659FF00D9927729FB00DE11DB8
:100BA000F91F639FB00DE11DF91FBD01CF01112495
:100BB0000895AA1BBB1B51E107C0AA1FBB1FA617A4
:100BC000B70710F0A61BB70B881F991F5A95A9F7F6
:100BD00080959095BC01CD010895A1E21A2EAA1B23
:100BE000BB1BFD010DC0AA1FBB1FEE1FFF1FA217DD
:100BF000B307E407F50720F0A21BB30BE40BF50BDA
:100C0000661F771F881F991F1A9469F76095709562
:100C1000809590959B01AC01BD01CF01089597FB94
:100C2000092E05260ED057FD04D0D7DF0AD0001CB0
:100C300038F450954095309521953F4F4F4F5F4F79
:100C40000895F6F790958095709561957F4F8F4F39
:040C50009F4F089515
:100C54000900000000010000021500040D00050356
:100C6400000618000806000911000A11001001000E
:100C7400110200121500141100151700161800189F
:100C84000700191A001A090020010021020022128B
:100C940000240D0025140026120028130029140036
:080CA4002ABAFF00004600001F
:00000001FF
